 KbdUs

 Timestamp is 4fb04cb3 (Mon May 14 12:07:15 2012)

 Preferred load address is 10000000

 Start         Length     Name                   Class
 0001:00000000 00000004H .CRT$XCA                CODE
 0001:00000004 00000004H .CRT$XCZ                CODE
 0001:00000008 00000004H .CRT$XIA                CODE
 0001:0000000c 00000004H .CRT$XIZ                CODE
 0001:00000010 00000004H .CRT$XPA                CODE
 0001:00000014 00000004H .CRT$XPZ                CODE
 0001:00000018 00000004H .CRT$XTA                CODE
 0001:0000001c 00000004H .CRT$XTZ                CODE
 0001:00000020 00000494H .rdata                  CODE
 0001:000004b4 00000022H .rdata$debug            CODE
 0001:000004d8 000045fcH .text                   CODE
 0001:00004ad4 000000ccH .xdata                  CODE
 0001:00004ba0 0000003cH .idata$2                CODE
 0001:00004bdc 00000014H .idata$3                CODE
 0001:00004bf0 00000124H .idata$4                CODE
 0001:00004d14 0000007eH .idata$6                CODE
 0001:00004da0 00000232H .edata                  CODE
 0002:00000000 00000124H .idata$5                DATA
 0002:00000128 000003f4H .data                   DATA
 0002:00000520 000004c8H .bss                    DATA
 0003:00000000 00000260H .pdata                  DATA

  Address         Publics by Value              Rva+Base       Lib:Object

 0000:00000000       ___safe_se_handler_count   00000000     <absolute>
 0000:00000000       ___safe_se_handler_table   00000000     <absolute>
 0001:00000000       __xc_a                     10001000     corelib0:crt0init.obj
 0001:00000004       __xc_z                     10001004     corelib0:crt0init.obj
 0001:00000008       __xi_a                     10001008     corelib0:crt0init.obj
 0001:0000000c       __xi_z                     1000100c     corelib0:crt0init.obj
 0001:00000010       __xp_a                     10001010     corelib0:crt0init.obj
 0001:00000014       __xp_z                     10001014     corelib0:crt0init.obj
 0001:00000018       __xt_a                     10001018     corelib0:crt0init.obj
 0001:0000001c       __xt_z                     1000101c     corelib0:crt0init.obj
 0001:00000360       ??_C@_17LIMMJKCA@?$AAK?$AAB?$AAD?$AA?$AA@ 10001360     LayoutManager:LayMgr.obj
 0001:00000368       ??_C@_1DA@FKJDDCGN@?$AAK?$AAe?$AAy?$AAb?$AAo?$AAa?$AAr?$AAd?$AA?5?$AAL?$AAa?$AAy?$AAo?$AAu?$AAt?$AA?2?$AAP?$AAr?$AAe?$AAl?$AAo?$AAa?$AAd?$AA?$AA@ 10001368     LayoutManager:LayMgr.obj
 0001:00000398       ??_C@_15EFLNJKHH@?$AA?$CF?$AAu?$AA?$AA@ 10001398     LayoutManager:LayMgr.obj
 0001:000003a0       ??_C@_19NGFMKOON@?$AA?$CF?$AA0?$AA8?$AAX?$AA?$AA@ 100013a0     LayoutManager:LayMgr.obj
 0001:000003ac       ??_C@_1CA@GLIJBCFK@?$AAK?$AAe?$AAy?$AAb?$AAo?$AAa?$AAr?$AAd?$AA?5?$AAL?$AAa?$AAy?$AAo?$AAu?$AAt?$AA?$AA@ 100013ac     LayoutManager:LayMgr.obj
 0001:000003cc       ??_C@_1M@LLCLNBHO@?$AA?$CF?$AAs?$AA_?$AA?$CF?$AAs?$AA?$AA@ 100013cc     LayoutManager:LayMgr.obj
 0001:000003d8       ??_C@_1EC@PDDNOLEO@?$AAK?$AAe?$AAr?$AAn?$AAe?$AAl?$AA?5?$AAP?$AAr?$AAo?$AAf?$AAi?$AAl?$AAe?$AAr?$AA?5?$AAm?$AAo?$AAd?$AAe?$AA?3?$AA?5?$AAB?$AAu?$AAf?$AAf?$AAe?$AAr?$AAe?$AAd?$AA?$AN?$AA?6@ 100013d8     LayoutManager:profiler.obj
 0001:0000041c       ??_C@_1DM@LDFFLEGF@?$AAK?$AAe?$AAr?$AAn?$AAe?$AAl?$AA?5?$AAP?$AAr?$AAo?$AAf?$AAi?$AAl?$AAe?$AAr?$AA?5?$AAm?$AAo?$AAd?$AAe?$AA?3?$AA?5?$AAC?$AAe?$AAL?$AAo?$AAg?$AA?$AN?$AA?6?$AA?$AA@ 1000141c     LayoutManager:profiler.obj
 0001:00000458       ??_C@_1EG@OLMAKGJN@?$AAK?$AAe?$AAr?$AAn?$AAe?$AAl?$AA?5?$AAP?$AAr?$AAo?$AAf?$AAi?$AAl?$AAe?$AAr?$AA?5?$AAm?$AAo?$AAd?$AAe?$AA?3?$AA?5?$AAU?$AAn?$AAb?$AAu?$AAf?$AAf?$AAe?$AAr?$AAe?$AAd@ 10001458     LayoutManager:profiler.obj
 0001:000004a0       ??_C@_1BE@MPEJEKEH@?$AAK?$AAP?$AAP?$AAL?$AAa?$AAy?$AAo?$AAu?$AAt?$AA?$AA@ 100014a0     Keypad_mx25_topaz_v1:kbd.obj
 0001:000004d8       KPPLayout                  100014d8 f   BSPKeypad:bspkeypad.obj
 0001:00000510       ?BSPKppIsWakeUpSource@@YAHXZ 10001510 f   BSPKeypad:bspkeypad.obj
 0001:00000518       ?BSPKppRegInit@@YAHXZ      10001518 f   BSPKeypad:bspkeypad.obj
 0001:00000bc8       ?BSPKppPowerOn@@YAHXZ      10001bc8 f   BSPKeypad:bspkeypad.obj
 0001:00000c3c       ?BSPKppPowerOff@@YAHXZ     10001c3c f   BSPKeypad:bspkeypad.obj
 0001:00000cd8       ?BSPKPPGetScanCodes@@YAIQAIQAH@Z 10001cd8 f   BSPKeypad:bspkeypad.obj
 0001:00000de4       IL_00000409                10001de4 f   InputLang_0409:IL_0409.obj
 0001:0000159c       KeybdDriverInitStates      1000259c f   LayoutManager:LayMgr.obj
 0001:000015c4       KeybdDriverGetInfo         100025c4 f   LayoutManager:LayMgr.obj
 0001:00001764       KeybdDriverSetMode         10002764 f   LayoutManager:LayMgr.obj
 0001:00001828       KeybdDriverPowerHandler    10002828 f   LayoutManager:LayMgr.obj
 0001:00001a44       ?KeybdEventThreadProc@@YAKPAX@Z 10002a44 f   LayoutManager:LayMgr.obj
 0001:00001ccc       ?KeybdEventCallback@@YAXIIH@Z 10002ccc f   LayoutManager:LayMgr.obj
 0001:00002688       ?GetKeyboardProcAddr@@YAP6AHXZPAUHINSTANCE__@@PBG@Z 10003688 f   LayoutManager:LayMgr.obj
 0001:000030e8       KeybdDriverInitializeEx    100040e8 f   LayoutManager:LayMgr.obj
 0001:00003388       LayoutMgrGetKeyboardType   10004388 f   LayoutManager:LayMgr.obj
 0001:0000340c       LayoutMgrGetKeyboardLayout 1000440c f   LayoutManager:LayMgr.obj
 0001:00003450       LayoutMgrGetKeyboardLayoutName 10004450 f   LayoutManager:LayMgr.obj
 0001:000034c8       LayoutMgrGetKeyboardLayoutList 100044c8 f   LayoutManager:LayMgr.obj
 0001:00003714       LayoutMgrLoadKeyboardLayout 10004714 f   LayoutManager:LayMgr.obj
 0001:0000395c       LayoutMgrActivateKeyboardLayout 1000495c f   LayoutManager:LayMgr.obj
 0001:000039d8       DllMain                    100049d8 f   LayoutManager:LayMgr.obj
 0001:000039f0       KeybdDriverVKeyToUnicode   100049f0 f   LayoutManager:LayMgr.obj
 0001:00003d28       KeybdDriverMapVirtualKey   10004d28 f   LayoutManager:LayMgr.obj
 0001:00003edc       ?DoProfilerKey@@YAHG@Z     10004edc f   LayoutManager:profiler.obj
 0001:00003fb0       Sleep                      10004fb0 f   coredll:COREDLL.dll
 0001:00003fc0       GetTickCount               10004fc0 f   coredll:COREDLL.dll
 0001:00003fd0       LeaveCriticalSection       10004fd0 f   coredll:COREDLL.dll
 0001:00003fe0       EnterCriticalSection       10004fe0 f   coredll:COREDLL.dll
 0001:00003ff0       InitializeCriticalSection  10004ff0 f   coredll:COREDLL.dll
 0001:00004000       EventModify                10005000 f   coredll:COREDLL.dll
 0001:00004010       SetLastError               10005010 f   coredll:COREDLL.dll
 0001:00004020       DeviceIoControl            10005020 f   coredll:COREDLL.dll
 0001:00004030       keybd_event                10005030 f   coredll:COREDLL.dll
 0001:00004040       WaitForSingleObject        10005040 f   coredll:COREDLL.dll
 0001:00004050       SetThreadPriority          10005050 f   coredll:COREDLL.dll
 0001:00004060       WaitForMultipleObjects     10005060 f   coredll:COREDLL.dll
 0001:00004070       StopDeviceNotifications    10005070 f   coredll:COREDLL.dll
 0001:00004080       GetLastError               10005080 f   coredll:COREDLL.dll
 0001:00004090       CloseHandle                10005090 f   coredll:COREDLL.dll
 0001:000040a0       CreateFileW                100050a0 f   coredll:COREDLL.dll
 0001:000040b0       ReadMsgQueue               100050b0 f   coredll:COREDLL.dll
 0001:000040c0       RequestDeviceNotifications 100050c0 f   coredll:COREDLL.dll
 0001:000040d0       CreateMsgQueue             100050d0 f   coredll:COREDLL.dll
 0001:000040e0       RegOpenKeyExW              100050e0 f   coredll:COREDLL.dll
 0001:000040f0       RegCloseKey                100050f0 f   coredll:COREDLL.dll
 0001:00004100       RegQueryValueExW           10005100 f   coredll:COREDLL.dll
 0001:00004110       StringCchCopyW             10005110 f   coredll:COREDLL.dll
 0001:00004120       GetProcAddressW            10005120 f   coredll:COREDLL.dll
 0001:00004130       FreeLibrary                10005130 f   coredll:COREDLL.dll
 0001:00004140       LoadLibraryW               10005140 f   coredll:COREDLL.dll
 0001:00004150       RegEnumValueW              10005150 f   coredll:COREDLL.dll
 0001:00004160       LocalFree                  10005160 f   coredll:COREDLL.dll
 0001:00004170       LocalAlloc                 10005170 f   coredll:COREDLL.dll
 0001:00004180       DeleteCriticalSection      10005180 f   coredll:COREDLL.dll
 0001:00004190       CreateThread               10005190 f   coredll:COREDLL.dll
 0001:000041a0       CreateEventW               100051a0 f   coredll:COREDLL.dll
 0001:000041b0       CeSafeCopyMemory           100051b0 f   coredll:COREDLL.dll
 0001:000041c0       RegDeleteKeyW              100051c0 f   coredll:COREDLL.dll
 0001:000041d0       RegSetValueExW             100051d0 f   coredll:COREDLL.dll
 0001:000041e0       RegCreateKeyExW            100051e0 f   coredll:COREDLL.dll
 0001:000041f0       StringCchLengthW           100051f0 f   coredll:COREDLL.dll
 0001:00004200       DisableThreadLibraryCalls  10005200 f   coredll:COREDLL.dll
 0001:00004210       NKDbgPrintfW               10005210 f   coredll:COREDLL.dll
 0001:00004220       ProfileStart               10005220 f   coredll:COREDLL.dll
 0001:00004230       ProfileStop                10005230 f   coredll:COREDLL.dll
 0001:00004240       MmMapIoSpace               10005240 f   ceddk:CEDDK.dll
 0001:00004250       DDKClockSetGatingMode      10005250 f   cspddk:CSPDDK.dll
 0001:00004260       DDKIomuxSetPadConfig       10005260 f   cspddk:CSPDDK.dll
 0001:00004270       DDKIomuxSetPinMux          10005270 f   cspddk:CSPDDK.dll
 0001:00004280       DDKClockGetGatingMode      10005280 f   cspddk:CSPDDK.dll
 0001:00004394       _DllMainCRTStartup         10005394 f   corelib0:pegdmain.obj
 0001:000043c4       __GSHandlerCheckCommon     100053c4 f   corelib0:gshandler.obj
 0001:00004400       __GSHandlerCheck           10005400 f   corelib0:gshandler.obj
 0001:00004424       __security_init_cookie     10005424 f   corelib0:seccinit.obj
 0001:00004480       __security_check_cookie    10005480 f   corelib0:armsecgs.obj
 0001:00004494       __gsfailure                10005494 f   corelib0:armsecgs.obj
 0001:000044d8       __GSHandlerCheck_SEH       100054d8 f   corelib0:gshandlerseh.obj
 0001:00004624       _cexit                     10005624 f   corelib0:cexit.obj
 0001:00004640       _initterm                  10005640 f   corelib0:crt0dat.obj
 0001:00004674       _cinit                     10005674 f   corelib0:crt0dat.obj
 0001:000046a8       memcpy                     100056a8 f   corelib1:COREDLL.dll
 0001:000046b8       memset                     100056b8 f   corelib1:COREDLL.dll
 0001:000046c8       wcsrchr                    100056c8 f   corelib1:COREDLL.dll
 0001:000046d8       wcsstr                     100056d8 f   corelib1:COREDLL.dll
 0001:000046e8       __C_specific_handler       100056e8 f   corelib1:COREDLL.dll
 0001:000046f8       _snwprintf                 100056f8 f   corelib1:COREDLL.dll
 0001:00004708       wcstoul                    10005708 f   corelib1:COREDLL.dll
 0001:00004718       wcscpy                     10005718 f   corelib1:COREDLL.dll
 0001:00004728       _wcsicmp                   10005728 f   corelib1:COREDLL.dll
 0001:00004738       _wcslwr                    10005738 f   corelib1:COREDLL.dll
 0001:00004748       wcsncat                    10005748 f   corelib1:COREDLL.dll
 0001:00004758       wcsncpy                    10005758 f   corelib1:COREDLL.dll
 0001:00004768       wcsncmp                    10005768 f   corelib1:COREDLL.dll
 0001:00004778       towlower                   10005778 f   corelib1:COREDLL.dll
 0001:00004788       _XcptFilter                10005788 f   corelib1:COREDLL.dll
 0001:00004798       __security_gen_cookie2     10005798 f   corelib1:COREDLL.dll
 0001:000047a8       __report_gsfailure         100057a8 f   corelib1:COREDLL.dll
 0001:000047b8       free                       100057b8 f   corelib1:COREDLL.dll
 0001:000047c8       ?CSPKppGetIrq@@YAIXZ       100057c8 f   Keypad_mx25_topaz_v1:soc_keypad.obj
 0001:000047d0       ?CSPKppGetBaseRegAddr@@YAIXZ 100057d0 f   Keypad_mx25_topaz_v1:soc_keypad.obj
 0001:000047dc       InterlockedExchange        100057dc f   coredll:COREDLL.dll
 0001:000047ec       TerminateProcess           100057ec f   coredll:COREDLL.dll
 0001:00004810       ?KPP_Entry@@YAHIP6AXIIH@ZPAPAUtagKEYBD_PDD@@@Z 10005810 f   Keypad_mx25_topaz_v1:kbd.obj
 0001:00004844       ?KeybdPdd_PowerHandler@@YAXH@Z 10005844 f   Keypad_mx25_topaz_v1:keypad.obj
 0001:00004880       ?KppIsrThreadProc@@YAHPAX@Z 10005880 f   Keypad_mx25_topaz_v1:keypad.obj
 0001:000048e4       ?KppIsrThreadStart@@YAHXZ  100058e4 f   Keypad_mx25_topaz_v1:keypad.obj
 0001:00004930       ?KppInitialize@@YAHXZ      10005930 f   Keypad_mx25_topaz_v1:keypad.obj
 0001:00004a28       ?KeybdIstLoop@@YAHPAUtagKEYBD_IST@@@Z 10005a28 f   KeybdIst:KeybdIst.obj
 0001:00004aa4       InterruptInitialize        10005aa4 f   coredll:COREDLL.dll
 0001:00004ab4       KernelIoControl            10005ab4 f   coredll:COREDLL.dll
 0001:00004ac4       InterruptDone              10005ac4 f   coredll:COREDLL.dll
 0001:00004ba0       __IMPORT_DESCRIPTOR_COREDLL 10005ba0     coredll:COREDLL.dll
 0001:00004bb4       __IMPORT_DESCRIPTOR_CEDDK  10005bb4     ceddk:CEDDK.dll
 0001:00004bc8       __IMPORT_DESCRIPTOR_CSPDDK 10005bc8     cspddk:CSPDDK.dll
 0001:00004bdc       __NULL_IMPORT_DESCRIPTOR   10005bdc     coredll:COREDLL.dll
 0002:00000000       __imp_MmMapIoSpace         10006000     ceddk:CEDDK.dll
 0002:00000004       \177CEDDK_NULL_THUNK_DATA  10006004     ceddk:CEDDK.dll
 0002:00000008       __imp_LeaveCriticalSection 10006008     coredll:COREDLL.dll
 0002:0000000c       __imp_EnterCriticalSection 1000600c     coredll:COREDLL.dll
 0002:00000010       __imp_InitializeCriticalSection 10006010     coredll:COREDLL.dll
 0002:00000014       __imp_EventModify          10006014     coredll:COREDLL.dll
 0002:00000018       __imp_SetLastError         10006018     coredll:COREDLL.dll
 0002:0000001c       __imp_DeviceIoControl      1000601c     coredll:COREDLL.dll
 0002:00000020       __imp_keybd_event          10006020     coredll:COREDLL.dll
 0002:00000024       __imp_WaitForSingleObject  10006024     coredll:COREDLL.dll
 0002:00000028       __imp_SetThreadPriority    10006028     coredll:COREDLL.dll
 0002:0000002c       __imp_WaitForMultipleObjects 1000602c     coredll:COREDLL.dll
 0002:00000030       __imp_StopDeviceNotifications 10006030     coredll:COREDLL.dll
 0002:00000034       __imp_GetLastError         10006034     coredll:COREDLL.dll
 0002:00000038       __imp_CloseHandle          10006038     coredll:COREDLL.dll
 0002:0000003c       __imp_CreateFileW          1000603c     coredll:COREDLL.dll
 0002:00000040       __imp_ReadMsgQueue         10006040     coredll:COREDLL.dll
 0002:00000044       __imp_RequestDeviceNotifications 10006044     coredll:COREDLL.dll
 0002:00000048       __imp_CreateMsgQueue       10006048     coredll:COREDLL.dll
 0002:0000004c       __imp_RegOpenKeyExW        1000604c     coredll:COREDLL.dll
 0002:00000050       __imp_RegCloseKey          10006050     coredll:COREDLL.dll
 0002:00000054       __imp_GetTickCount         10006054     coredll:COREDLL.dll
 0002:00000058       __imp_StringCchCopyW       10006058     coredll:COREDLL.dll
 0002:0000005c       __imp_GetProcAddressW      1000605c     coredll:COREDLL.dll
 0002:00000060       __imp_FreeLibrary          10006060     coredll:COREDLL.dll
 0002:00000064       __imp_LoadLibraryW         10006064     coredll:COREDLL.dll
 0002:00000068       __imp_RegEnumValueW        10006068     coredll:COREDLL.dll
 0002:0000006c       __imp_LocalFree            1000606c     coredll:COREDLL.dll
 0002:00000070       __imp_LocalAlloc           10006070     coredll:COREDLL.dll
 0002:00000074       __imp_DeleteCriticalSection 10006074     coredll:COREDLL.dll
 0002:00000078       __imp_CreateThread         10006078     coredll:COREDLL.dll
 0002:0000007c       __imp_CreateEventW         1000607c     coredll:COREDLL.dll
 0002:00000080       __imp_CeSafeCopyMemory     10006080     coredll:COREDLL.dll
 0002:00000084       __imp_RegDeleteKeyW        10006084     coredll:COREDLL.dll
 0002:00000088       __imp_RegSetValueExW       10006088     coredll:COREDLL.dll
 0002:0000008c       __imp_RegCreateKeyExW      1000608c     coredll:COREDLL.dll
 0002:00000090       __imp_StringCchLengthW     10006090     coredll:COREDLL.dll
 0002:00000094       __imp_DisableThreadLibraryCalls 10006094     coredll:COREDLL.dll
 0002:00000098       __imp_NKDbgPrintfW         10006098     coredll:COREDLL.dll
 0002:0000009c       __imp_ProfileStart         1000609c     coredll:COREDLL.dll
 0002:000000a0       __imp_ProfileStop          100060a0     coredll:COREDLL.dll
 0002:000000a4       __imp_RegQueryValueExW     100060a4     coredll:COREDLL.dll
 0002:000000a8       __imp_Sleep                100060a8     coredll:COREDLL.dll
 0002:000000ac       __imp_KernelIoControl      100060ac     coredll:COREDLL.dll
 0002:000000b0       __imp_InterruptInitialize  100060b0     coredll:COREDLL.dll
 0002:000000b4       __imp_TerminateProcess     100060b4     coredll:COREDLL.dll
 0002:000000b8       __imp_InterlockedExchange  100060b8     coredll:COREDLL.dll
 0002:000000bc       __imp_memcpy               100060bc     corelib1:COREDLL.dll
 0002:000000c0       __imp_memset               100060c0     corelib1:COREDLL.dll
 0002:000000c4       __imp_wcsrchr              100060c4     corelib1:COREDLL.dll
 0002:000000c8       __imp_wcsstr               100060c8     corelib1:COREDLL.dll
 0002:000000cc       __imp___C_specific_handler 100060cc     corelib1:COREDLL.dll
 0002:000000d0       __imp___rt_udiv            100060d0     corelib1:COREDLL.dll
 0002:000000d4       __imp__snwprintf           100060d4     corelib1:COREDLL.dll
 0002:000000d8       __imp_wcstoul              100060d8     corelib1:COREDLL.dll
 0002:000000dc       __imp_wcscpy               100060dc     corelib1:COREDLL.dll
 0002:000000e0       __imp__wcsicmp             100060e0     corelib1:COREDLL.dll
 0002:000000e4       __imp__wcslwr              100060e4     corelib1:COREDLL.dll
 0002:000000e8       __imp_wcsncat              100060e8     corelib1:COREDLL.dll
 0002:000000ec       __imp_wcsncpy              100060ec     corelib1:COREDLL.dll
 0002:000000f0       __imp_wcsncmp              100060f0     corelib1:COREDLL.dll
 0002:000000f4       __imp_towlower             100060f4     corelib1:COREDLL.dll
 0002:000000f8       __imp__XcptFilter          100060f8     corelib1:COREDLL.dll
 0002:000000fc       __imp___security_gen_cookie2 100060fc     corelib1:COREDLL.dll
 0002:00000100       __imp___report_gsfailure   10006100     corelib1:COREDLL.dll
 0002:00000104       __imp_free                 10006104     corelib1:COREDLL.dll
 0002:00000108       __imp_InterruptDone        10006108     coredll:COREDLL.dll
 0002:0000010c       \177COREDLL_NULL_THUNK_DATA 1000610c     coredll:COREDLL.dll
 0002:00000110       __imp_DDKIomuxSetPinMux    10006110     cspddk:CSPDDK.dll
 0002:00000114       __imp_DDKIomuxSetPadConfig 10006114     cspddk:CSPDDK.dll
 0002:00000118       __imp_DDKClockSetGatingMode 10006118     cspddk:CSPDDK.dll
 0002:0000011c       __imp_DDKClockGetGatingMode 1000611c     cspddk:CSPDDK.dll
 0002:00000120       \177CSPDDK_NULL_THUNK_DATA 10006120     cspddk:CSPDDK.dll
 0002:000004fc       __security_cookie          100064fc     corelib0:seccinit.obj
 0002:00000500       __security_cookie_complement 10006500     corelib0:seccinit.obj
 0002:00000504       ?g_rgpfnPddEntries@@3PAP6AHIP6AXIIH@ZPAPAUtagKEYBD_PDD@@@ZA 10006504     PddList_common_topaz_v1:pddlist.obj
 0002:00000668       ?g_csEventCallback@@3UCRITICAL_SECTION@@A 10006668     LayoutManager:LayMgr.obj
 0002:000009c0       _exitflag                  100069c0     corelib0:cexit.obj
 0002:000009c4       ?v_uiPddId@@3IA            100069c4     Keypad_mx25_topaz_v1:kbd.obj
 0002:000009c8       ?v_pfnKeybdEvent@@3P6AXIIH@ZA 100069c8     Keypad_mx25_topaz_v1:kbd.obj
 0002:000009cc       ?g_dwSysIntr_Keybd@@3KA    100069cc     Keypad_mx25_topaz_v1:keypad.obj
 0002:000009d0       ?g_hevInterrupt@@3PAXA     100069d0     Keypad_mx25_topaz_v1:keypad.obj
 0002:000009d8       __onexitend                100069d8     <common>
 0002:000009dc       __onexitbegin              100069dc     <common>
 0002:000009e0       g_pcsExit                  100069e0     <common>
 0002:000009e4       _pRawDllMain               100069e4     <common>

 entry point at        0001:00004394

 Static symbols

 0001:0000076c       ?KppScanSequence@@YAIQAIQAHH@Z 1000176c f   BSPKeypad:bspkeypad.obj
 0001:00000e1c       ?ScanCodeToVKey@@YAHIPAPAUScanCodeToVKeyData@@IPAI@Z 10001e1c f   LayoutManager:LayMgr.obj
 0001:00000ea8       ?ProcessDeadKeys@@YAIPAGPBU_DEADKEY@@GPAIII@Z 10001ea8 f   LayoutManager:LayMgr.obj
 0001:00000f44       ?ProcessLigature@@YAIPAUtagINPUT_LANGUAGE_INFO@@IIGPAII@Z 10001f44 f   LayoutManager:LayMgr.obj
 0001:00001058       ?GetCharacters@@YAIPAUtagINPUT_LANGUAGE_INFO@@PBU_VK_TO_WCHAR_TABLE@@PBU_VK_TO_WCHARS1@@GIPAII@Z 10002058 f   LayoutManager:LayMgr.obj
 0001:0000120c       ?VKeyToUnicode@@YAIPAUtagINPUT_LANGUAGE_INFO@@IIPAII@Z 1000220c f   LayoutManager:LayMgr.obj
 0001:000013ac       ?AltNumKeyEvent@@YAHIIPAI0@Z 100023ac f   LayoutManager:LayMgr.obj
 0001:00001700       ?BroadcastToKeyboards@@YAXKPAXK@Z 10002700 f   LayoutManager:LayMgr.obj
 0001:000018ac       ?CallDLRemapFn@@YAIP6AIPBU_KEYBD_EVENT@@IPAU1@I@Z0I1I@Z 100028ac f   LayoutManager:LayMgr.obj
 0001:00001914       ?SendRemappedEvent@@YAXIIIHPAUtagDEVICE_LAYOUT_INFO@@@Z 10002914 f   LayoutManager:LayMgr.obj
 0001:00001d48       ?KbdNotificationThread@@YAKPAX@Z 10002d48 f   LayoutManager:LayMgr.obj
 0001:00002058       ?GetPreloadInputMethodKey@@YAHIPAPAUHKEY__@@@Z 10003058 f   LayoutManager:LayMgr.obj
 0001:00002124       ?GetPreloadInputMethodName@@YAHIPAG@Z 10003124 f   LayoutManager:LayMgr.obj
 0001:000021b8       ?GetInputMethodInfo@@YAHPBGPAUtagINPUT_LANGUAGE_INFO@@@Z 100031b8 f   LayoutManager:LayMgr.obj
 0001:00002310       ?GetDefaultInputMethodName@@YAHPAG@Z 10003310 f   LayoutManager:LayMgr.obj
 0001:00002468       ?GenerateModifierToShiftTable@@YAHPAUtagINPUT_LANGUAGE_INFO@@@Z 10003468 f   LayoutManager:LayMgr.obj
 0001:00002540       ?GetImeKeyboardLayout@@YAPAUHKL__@@PAU1@@Z 10003540 f   LayoutManager:LayMgr.obj
 0001:0000270c       ?SetInputLanguage@@YAHPAUHKL__@@PAPAU1@@Z 1000370c f   LayoutManager:LayMgr.obj
 0001:00002a3c       ?DeviceLayoutMatchesPDD@@YAHPBG00GPAGK@Z 10003a3c f   LayoutManager:LayMgr.obj
 0001:00002c30       ?SelectDeviceLayout@@YAHPAGPAUtagKEYBD_PDD@@0K0K@Z 10003c30 f   LayoutManager:LayMgr.obj
 0001:00002e4c       ?SetDeviceLayout@@YAHPAUHKL__@@I@Z 10003e4c f   LayoutManager:LayMgr.obj
 0001:000035d4       ?IsLayoutLoaded@@YAHPBG@Z  100045d4 f   LayoutManager:LayMgr.obj
 0001:00004298       _DllMainCRTStartupHelper   10005298 f   corelib0:pegdmain.obj
 0001:00004528       doexit                     10005528 f   corelib0:cexit.obj
 0001:000047fc       ?KPP_PowerHandler@@YAXIH@Z 100057fc f   Keypad_mx25_topaz_v1:kbd.obj
 0001:00004868       ?KeybdPdd_GetEventEx2@@YAIIQAIQAH@Z 10005868 f   Keypad_mx25_topaz_v1:keypad.obj
